:1000000011C020C01FC01EC01DC01CC01BC01AC014
:1000100019C018C017C016C015C014C013C06E6F29
:100020006465200011241FBECFE5D1E0DEBFCDBF47
:1000300020E0A0E6B0E001C01D92A436B207E1F7CF
:1000400005D134C1DDCFDC01FA0110828C91862309
:10005000E9F782E28A95F1F700C085E48A95F1F725
:1000600000008C91862319F080818160808385E473
:100070008A95F1F700008C91862319F080818260C7
:10008000808385E48A95F1F700008C91862319F02E
:1000900080818460808385E48A95F1F700008C91EB
:1000A000862319F080818860808385E48A95F1F742
:1000B00000008C91862319F080818061808385E423
:1000C0008A95F1F700008C91862319F08081806277
:1000D000808385E48A95F1F700008C91862319F0DE
:1000E00080818064808385E48A95F1F700008C919B
:1000F000862319F080818068808385E48A95F1F7F2
:10010000000082E28A95F1F700C00895FC01908119
:10011000862F80959823908395E49A95F1F70000B7
:10012000908140FF02C0962B01C09823908395E4F4
:100130009A95F1F70000908141FF02C0962B01C013
:100140009823908395E49A95F1F70000908142FFFF
:1001500002C0962B01C09823908395E49A95F1F7FD
:100160000000908143FF02C0962B01C0982390832A
:1001700095E49A95F1F70000908144FF02C0962B18
:1001800001C09823908395E49A95F1F7000090813F
:1001900045FF02C0962B01C09823908395E49A9561
:1001A000F1F70000908146FF02C0962B01C0982312
:1001B000908395E49A95F1F7000047FF04C0808191
:1001C000862B808303C090819823908385E48A9551
:1001D000F1F700008081862B808395E49A95F1F7F2
:1001E000000085E48A95F1F700000895CF93DF932E
:1001F000EA011092630010926200E0916200F091B7
:100200006300EC0FFD1F44914093610060E188E3BF
:1002100090E07CDF80916200909163000196909362
:10022000630080936200809161008111E6CFDF91CD
:10023000CF910895C0982FEF80E792E02150804041
:100240009040E1F700C00000C09A089580E886BDA4
:1002500016BCC49ABC98C09AB89A40E650E068E0D0
:1002600086E390E0F0DEE6DF809160008033A9F75E
:10027000BC9A4EE150E060E188E390E0B7DF409146
:10028000600060E188E390E041DF4AE060E188E3FC
:1002900090E03CDF2FEF80E792E0215080409040DB
:1002A000E1F700C00000C6DFBC98D7CFF894FFCFBD
:00000001FF
